:1064F3000A2A2A2A2A2A2A2A2A2A2A2A2A2A2A2A19
:106503002A2A20CFE0F0E0ECE5F2F0FB20E0E4E023
:10651300EFF2E5F0E0202A2A2A2A2A2A2A2A2A2A1E
:106523002A2A2A2A2A2A2A2A0A00312E204D4143BE
:1065330020E0E4F0E5F13A202025303262783A2574
:10654300303262783A25303262783A2530326278D6
:106553003A25303262783A25303262780A00322E98
:1065630020495020E0E4F0E5F13A2020202562752F
:106573002E2562752E2562752E2562750A00332E2F
:1065830020D8EBFEE73A202020202020202562752A
:106593002E2562752E2562752E2562750A00342E0E
:1065A30020CCE0F1EAE020F1E5F2E83A202562753B
:1065B3002E2562752E2562752E2562750A00352EED
:1065C30020495020E0E4F0E5F120F1E5F0E2E5F0C8
:1065D300E0313A202562752E2562752E2562752ECF
:1065E3002562750A00362E20495020E0E4F0E5F1DB
:1065F30020F1E5F0E2E5F0E0323A202562752E2540
:1066030062752E2562752E2562750A00302E20CA0A
:10661300EBFEF720E4EEF1F2F3EFE03A2025730A04
:10662300000AC7C0CFC8D1DC20466C6173680A007A
:106633000AC7E0EFE8F1FC20E7E0E2E5F0F8E5ED7A
:10664300E0210A00082008000A53696E636F6D4950
:1066530050205665722E20332E30204343202827A6
:106663002B2B2B272DE2F5EEE420E220EAEEEDF4CE
:10667300E8E3F3F0E0F2EEF029000A3E20CAEEED83
:10668300F4E8E3F3F0E0F6E8EEEDEDFBE920F0E506
:10669300E6E8EC0A0A00203C493E20203A20CFEEEF
:1066A300EAE0E7E0F2FC20EFE0F0E0ECE5F2F0FBFB
:1066B3000A00203C536E3E203A20C7E0E4E0F2FC9F
:1066C30020EFE0F0E0ECE5F2F020276E270A00204F
:1066D3003C4B3E20203A20C7E0E3F0F3E7E8F2FC2E
:1066E30020EDEEE2F3FE20EAEEEDF42E20E8E720C3
:1066F300F4E0E9EBE00A00203C443E20203A20D0BD
:10670300E0F1EFE5F7E0F2E0F2FC20EDEEE2F3FE7C
:1067130020EAEEEDF42E0A00203C573E20203A20DA
:10672300C7E0EFE8F1E0F2FC20E8E7ECE5EDE5EDAA
:10673300E8FF0A00203C4C3E20203A20C7E0E3F06B
:10674300F3E7E8F2FC20EFF0EEE3F0E0ECECF32803
:10675300584D4F44454D290A00203C453E20203AE0
:1067630020C2FBF5EEE40A003E20C2E2E5E4E8F2D3
:10677300E520EAEEECE0EDE4F33A20000AC2E2E5BC
:10678300E4E8F2E520274D414320E0E4F0E5F15B46
:106793002562645D273A202530326278202D3E0041
:1067A30078000AC2E2E5E4E8F2E52027495020E058
:1067B300E4E0EFF2E5F0E05B2562645D273A202533
:1067C3006275202D3E0075000AC2E2E5E4E8F2E5B9
:1067D3002027D8EBFEE75B2562645D273A2025621C
:1067E30075202D3E000AC2E2E5E4E8F2E52027CC5D
:1067F300E0F1EAF3D1E5F2E85B2562645D273A2034
:10680300256275202D3E000AC2E2E5E4E8F2E520A8
:1068130027495020F1E5F0E2E5F0E0315B256264C1
:106823005D273A20256275202D3E000AC2E2E5E489
:10683300E8F2E52027495020F1E5F0E2E5F0E03207
:106843005B2562645D273A20256275202D3E000A90
:10685300C2E2E5E4E8F2E520EAEBFEF720E4EEF13C
:10686300F2F3EFE028E4EE203720F1E8ECE2293AF6
:106873000A2D3E000A204572726F72210A000AC86F
:10688300C4C5D220C7C0CFC8D1DC2120C6C4C8D25A
:10689300C521000AC7C0CFC8D1DC20C7C0C2C5D03C
:1068A300D8C5CDC0210A000A20000ACA20EFF0E8AB
:1068B300E5ECF320E3EEF2EEE2210A00C7E0EFF3AA
:1068C300F1F2E8F2E520EFE5F0E5E4E0F7F320424A
:1068D300494E20F4E0E9EBE020F120EFEEECEEF995
:1068E300FCFE20584D4F44454D0A000A454F5421A4
:1068F3000A000AD4E0E9EB20E7E0E3F0F3E6E5ED94
:10690300210A00CEF8E8E1EAE0210A000AD4E0E92E
:10691300EB20EFEEEBF3F7E5ED2120C7E0EFE8F135
:10692300FC20E220454550524F4D210A003C4D4189
:10693300433D003C4130313D003C4130323D003C61
:106943004130333D003C4130343D003C4130353D26
:10695300003C4130363D000ACAEEEDF4E8E3F3F0C3
:10696300E0F6E8FF20E7E0EFE8F1E0EDE0210A00E0
:10776200C2ADE4F5C9D2CDD2CCC2C9C2CAF5CDF5FB
:10777200CC75CBFF75CAB885CBCD85CACCD29ED28B
:0A7782009CD2CAC2ACC298C2992280
:077863003098FDAF99C298B7
:01786A0022FB
:06784900127863EFF52246
:08784F008F993099FDC29922C6
:10783900AE07BE0A057F0D12784FAF0612784F22A8
:1074B6007BFF7A6479F31269D57BFF7A65792D9023
:1074C60061A2E0F535A3E0F536A3E0F537A3E0F5D4
:1074D60038A3E0F539A3E0F53A1269D57BFF7A6562
:1074E60079619061A8E0F535A3E0F536A3E0F537BC
:1074F600A3E0F5381269D57BFF7A65798190619AA8
:10750600E0F535A3E0F536A3E0F537A3E0F538124C
:1075160069D57BFF7A6579A190619EE0F535A3E098
:10752600F536A3E0F537A3E0F5381269D57BFF7A87
:107536006579C19061B1E0F535A3E0F536A3E0F5D4
:1075460037A3E0F5381269D57BFF7A6579E8906153
:10755600B5E0F535A3E0F536A3E0F537A3E0F53859
:107566001269D57535017536617537CB7BFF7A663D
:05757600790F0269D548
:06757B008E298F2A8D2BE2
:10758100E4F530F531F52EF52FE52B60097BFF7A17
:107591006679241269D5E4F52CF52DE529C4F85452
:1075A100F0C868FEE52AC4540F48FFC3E52D9FE5E6
:1075B1002C9E5031AE30AF31AD07AC067B10AF2FF2
:1075C100AE2E12772E74102531F531E43530F530B9
:1075D1007410252FF52FE4352EF52E052DE52D7090
:1075E100BA052C80B6E529C4F854F0C868FEE52A2E
:1075F100C4540F48C4F8540FC868FFEEC454F0488F
:10760100FEC3E52A9FFFE5299EAC30AD31AB07AF44
:107611002FAE2E12772EE52B60097BFF7A66793328
:037621001269D516
:017624002243
:0473E9007E677FC973
:0473ED008E298F2A2C
:1073F100E4F52B7400252BF582E43460F583E4F089
:10740100052BE52BB408ECE4F52B127863EFF52C92
:10741100640A6005E52CB40D0F7400252BF582E498
:107421003460F583E4F08044E52CB40824E52BD3E3
:107431009400402F7BFF7A6679471269D5152B742A
:1074410000252BF582E43460F5837420F0152B8040
:10745100127400252BF582E43460F583E52CF0FFEE
:1074610012784F052BE52BC39408409EE52B700243
:10747100FF22852A82852983E493B4781E906000D7
:10748100E0FF1276FAEFC454F0FEC006906001E00E
:10749100FF1276FAD0E02FF50880177531007532AA
:1074A10000753300E4F5347B017A60790012710DC7
:0474B1008F087F01C0
:0174B50022B4
:10600300C2AFE58720E456907FFEE0B4FF047F0132
:1060130080027F00907FFDE0B4AA047E0180027EAF
:1060230000EE5FFF907FFFE0B455047E0180027EA7
:1060330000EE5F6019E4907FFDF0A3F0A3F0907F82
:10604300F0E0FEA3E0FF4E6005E4FD12757B7BFFED
:106053007A0079008B268A278928126FD85387EF15
:10606300127762C2987BFF7A66794B1269D53098B2
:106073000F7BFF7A0079008B268A278928126FD835
:10608300E4F525F523E523139290A290B39291E4CE
:10609300F5242098030264BE1278638F22E522B4AC
:1060A3002B0512784F0525E525C39403500302649D
:1060B300ADE4F523E5232401FFE433FE12781474E1
:1060C3009A2523F582E43461F583EFF00523E52374
:1060D300C3943F40DFE4F523E523247FFFE433FE4D
:1060E30012781474142523F582E43461F583EFF0F8
:1060F3000523E523C3948040DFE4906193F0E52515
:1061030070030264BE7BFF7A66797D1269D57BFFDB
:106113007A6679991269D57BFF7A6679B51269D562
:106123007BFF7A6679D21269D57BFF7A6679FA1298
:1061330069D57BFF7A67791B1269D57BFF7A67790B
:10614300371269D57BFF7A67795C1269D57BFF7A51
:1061530067796B1269D5127849E522126FB26466CA
:106163004463F745618F4964604B645A4C619553AE
:1061730063FD5764666463F765618F6964606B648C
:106183005A6C61957363FD77000061011274B60266
:106193006101127849E522126FB263423061B63170
:1061A30062073262463362853462C4356303360064
:1061B3000063EF9061A274FAF0A374CEF0A374CCE1
:1061C300F0752203E522C3940640030261017BFFBD
:1061D3007A67797F85223574A22522F582E43461BA
:1061E300F583E0F5361269D57E677FA31273EDEF71
:1061F300600E74A22522F582E43461F583E508F08C
:10620300052280C0E4F522E522C394044003026121
:10621300017BFF7A6779A585223574A82522F5824B
:10622300E43461F583E0F5361269D51273E9EF6062
:106233000E74A82522F582E43461F583E508F005A0
:106243002280C4E4F522E522C394044003026101E1
:106253007BFF7A6779CB852235749A2522F582E410
:106263003461F583E0F5361269D51273E9EF600EF8
:10627300749A2522F582E43461F583E508F005225A
:1062830080C4E4F522E522C3940440030261017B48
:10629300FF7A6779E8852235749E2522F582E434F6
:1062A30061F583E0F5361269D51273E9EF600E7478
:1062B3009E2522F582E43461F583E508F00522800A
:1062C300C4E4F522E522C3940440030261017BFF89
:1062D3007A68790A85223574B12522F582E434611E
:1062E300F583E0F5361269D51273E9EF600E74B1E8
:1062F3002522F582E43461F583E508F0052280C4A4
:10630300E4F522E522C3940440030261017BFF7A92
:1063130068792E85223574B52522F582E43461F53A
:1063230083E0F5361269D51273E9EF600E74B52573
:1063330022F582E43461F583E508F0052280C47B0D
:10634300FF7A6879521269D5E4F52374CB2523F5D6
:1063530082E43461F583E4F00523E523B408ECE437
:10636300F523127863EFF522640A6005E522B40D84
:106373000F74CB2523F582E43461F583E4F0804484
:10638300E522B40824E523D39400402F7BFF7A66EB
:1063930079471269D5152374CB2523F582E434613B
:1063A300F5837420F01523801274CB2523F582E442
:1063B3003461F583E522F0FF12784F0523E523C30B
:1063C3009408409E9061CBE064206003026101F574
:1063D30023E523C39408400302610174CB2523F50D
:1063E30082E43461F583E4F0052380E57BFF7A687A
:1063F3007977805DE4F5250261017BFF7A68798115
:106403001269D5E4F523E5232401FFE433FE749AEE
:106413002523F582E43461F583E0FD1277FF05233C
:10642300E523C3943F40DFE4F523E523247FFFE422
:1064330033FE74142523F582E43461F583E0FD1201
:1064430077FF0523E523C3948040DF7BFF7A6879D8
:10645300961269D50261011272B1026101126CCF09
:106463000261017BFF7A6879AA1269D5906194E48D
:10647300F0A374FFF0E4F523C3E52394D074809470
:10648300874003026101E522F47003026101E52202
:1064930070030261011277E98F2212784FE52264BB
:1064A300217003026101052380CEE525700D7BFF7A
:1064B300FAF98B26F527F528126FD87F147E001280
:1064C30077B20524E524C3941950030260957F2E07
:1064D30012784F0523E523C3940A50030260887B97
:1064E300FF7A0079008B268A278928126FD880FECD
:1077B200E4FDFCC3ED9FEC9E5014E4FBFA0BBB000E
:0E77C200010AEBF44A70F60DBD00010C80E5E3
:0177D0002296
:10778C00E4FF7E0374142EF582E43460F583E02F5D
:10779C00FF0EBE83EF74142EF582E43460F583E0A3
:0577AC00FEC3EF9EFF8B
:0177B10022B5
:1072B100752F60753017E4F52DF52EC2017BFF7A2D
:1072C1006879AD1269D57BFF7A6879BF1269D520DB
:1072D10098247F1512784FE4F529F52AC3E52A94FD
:1072E10020E529648094CE50E62098E3052AE52A1A
:1072F10070EA052980E6D200752C01E599B40409EC
:107301007BFF7A6879EE1269D53001030273C3C33A
:10731100E52E94C0E52D945D40030273C3E4F52B83
:1073210020983AE4F529F52AAE29AF2AEE3395E003
:10733100FDFCE47B407A9CF9F8D3126F36400D20B6
:10734100980A052AE52A70E0052980DC20980E308C
:1073510000047F0680027F1512784F80C3C298E532
:107361002B7009E599B40404D20180177414252BFC
:10737100F582E43460F583E599F0052BE52BC394A0
:1073810084409D12778CEF600A7F1512784FC200FE
:1073910002730AD200906015E0B52C1E052CAE2FA9
:1073A100AF30AD07AC067B80AF2EAE2D12772E74B9
:1073B10080252EF52EE4352DF52D7F0612784F020E
:1073C100730A7F2012784FE4F529F52A20981005D9
:1073D1002AE52A70020529B420F2E529B44EED7B95
:0873E100FF7A6879F50269D515
:1076FA00EFC39430400BEFD394395005EF24D0FFF9
:10770A0022EFC39461400BEFD394665005EF24A98E
:10771A00FF22EFC39441400BEFD394465005EF2468
:04772A00C9FF22224F
:1077E900906194E475F001126F20906194E0FEA31A
:0677F900E0FF12781422EB
:1077D1001277E91276FAEFC454F0FEC0061277E987
:0877E1001276FAD0E02FFF221E
:1076A5001277E9906000EFF01277E9906001EFF052
:1076B5001277E9906002EFF01277E9906003EFF03E
:1076C5001277E9906004EFF01277E9906005EFF02A
:1076D5001277E9906006EFF01277E9906007EFF016
:1076E500E4A3F0F531F532F533F5347B017A6079B1
:0576F5000012710D22DE
:047625008E2E8F2FE7
:10762900906194E4F0A374FFF01277E9EF6069F4D4
:107639006066852F82852E83E493B507EC7530014A
:10764900E52F2530F582E4352EF583E49360259006
:107659006195E02530FF906194E03400FE127814C2
:10766900E52F2530F582E4352EF583E493B507043B
:10767900053080CCE52F2530F582E4352EF583E4FD
:107689009370A6E53024FFFFE434FF9061948FF0F6
:0B769900126F207E007F0122E4FEFF44
:0176A40022C3
:106CCF007BFF7A6879AD1269D59061D9126F810017
:106CDF00000000E4F529F52A209841D3E52A940015
:106CEF00E529940040199061D9126F5DEF2401FFDF
:106CFF00E43EFEE43DFDE43CFC9061D9126F757FEC
:106D0F00E07E937D047C009061D9126F69D3126F7E
:106D1F004C40C57BFF7A697906026F1C9061D912CE
:106D2F006F81000000001278638F2DE52D643C60A9
:106D3F0011052AE52A70020529C394C0E529945D3F
:106D4F004096900000E52DF0752900752A01127804
:106D5F00638F2D852A82852983E52DF064216011AB
:106D6F00052AE52A70020529C394D0E52994074026
:106D7F00DD7BFF7A69790F1269D5E52A2401F52C9D
:106D8F00E43529F52BE4F529F52AC3E52A952CE5F9
:106D9F0029952B501EE4252AFFE5293401FE852A6B
:106DAF0082852983E0FD1277FF052AE52A70DB052E
:106DBF002980D77E697F30127625EF4E60301277AB
:106DCF00D19061A2EFF01277D19061A3EFF012771B
:106DDF00D19061A4EFF01277D19061A5EFF0127707
:106DEF00D19061A6EFF01277D19061A7EFF07E6995
:106DFF007F36127625EF4E60201277D19061A8EF83
:106E0F00F01277D19061A9EFF01277D19061AAEFCC
:106E1F00F01277D19061ABEFF07E697F3C1276254F
:106E2F00EF4E60201277D19061B1EFF01277D190D1
:106E3F0061B2EFF01277D19061B3EFF01277D1908A
:106E4F0061B4EFF07E697F42127625EF4E6020121B
:106E5F0077D19061B5EFF01277D19061B6EFF01264
:106E6F0077D19061B7EFF01277D19061B8EFF07EE4
:106E7F00697F48127625EF4E60201277D190619E80
:106E8F00EFF01277D190619FEFF01277D19061A060
:106E9F00EFF01277D19061A1EFF07E697F4E1276FD
:106EAF0025EF4E60201277D190619AEFF01277D1D3
:106EBF0090619BEFF01277D190619CEFF01277D138
:106ECF0090619DEFF07E697F54127625EF4E60083A
:106EDF001276A59061B9EFF0E4F529F52AE52A2499
:106EEF0001FFE43529FE749A252AF582E43461F511
:106EFF0083E0FD1277FF052AE52A70020529C39466
:106F0F0043E529940040D67BFF7A69795A1269D5F7
:016F1F00224F
:02772E008B329C
:10773000A2AF9202C2AF85A23353A2FE8E838F8284
:1077400005A28C838D827409127827E53253A2FE3C
:1077500043A22012782953A2DF8533A2A20292AF5E
:01776000FF29
:017761002205
:10781400438E2075D2028F828E83E0FFE4F5D2532B
:027824008EDFF5
:01782600223F
:1077FF00E5D220E0FB43D2028F828E83EDF075D26B
:05780F005063D250227D
:10782700F922C002C004C00612FFF0D006D004D06F
:0278370002222B
:03600000027857CC
:0C78570078FFE4F6D8FD7581450260035F
:106F2000C5F0F8A3E028F0C5F0F8E58215827002FC
:066F30001583E038F02299
:106F3600EB9FF5F0EA9E42F0E99D42F0EC6480C8D2
:066F460064809845F02272
:106F4C00EB9FF5F0EA9E42F0E99D42F0E89C45F09B
:016F5C002212
:0C6F5D00E0FCA3E0FDA3E0FEA3E0FF22A7
:0C6F6900E0F8A3E0F9A3E0FAA3E0FB22AB
:0C6F7500ECF0A3EDF0A3EEF0A3EFF0228F
:106F8100A8828583F0D083D082126F98126F9812F5
:106F91006F98126F98E473E493A3C583C5F0C5831A
:106FA100C8C582C8F0A3C583C5F0C583C8C582C85A
:016FB10022BD
:106FB200D083D082F8E4937012740193700DA3A36E
:106FC20093F8740193F5828883E473740293686082
:066FD200EFA3A3A380DF82
:066FD8008A838982E47344
:10697300E5412435F8E605412278323009027835BD
:10698300E475F001127093026FDE2002EB7F2ED2CA
:10699300028018EF540F2490D43440D4FF30060BF8
:1069A300EF24BFB41A0050032461FFE542600215CF
:1069B300420545E5457002054430090D7832E4751A
:1069C300F001127093EF0270240278397403D20934
:1069D3008003E4C209F5418B328A338934E4F542FA
:1069E300F544F545E54260077F201269AE80F575F1
:1069F30043FFC203C202C204C205C207C208C20ADD
:106A030012697CFF700D3009057F001269BFAF4525
:106A1300AE4422B4255FC2D5C20612697CFF24D0DE
:106A2300B40A00501A75F00A784230D50508B6FF4B
:106A33000106C6A426F620D5047002D20580D92407
:106A4300CFB41A00EF5004C2E5D206026BBFD203E3
:106A530080C6D20280C0D20480BCD2D580BAD2070D
:106A630080B47F201269AE2004077401B542004050
:106A7300F1126973FF1269AE0269E7D20AD2088084
:106A830095126973FB126973FA126973F94A4B70B1
:106A93000679907A6C7BFF20042EE542602A7E0003
:106AA3008E82758300126FF760060EEE654370F0F9
:106AB300C2D5EBC0E0EAC0E0E9C0E0EE126C06D05C
:106AC300E0F9D0E0FAD0E0FB126FDEFF60AAEBC082
:106AD300E0EAC0E0E9C0E01269AED0E02401F9D0F9
:106AE300E03400FAD0E0FBE5430460DCD543D98011
:106AF300877BFF7A6C7902D204809C7910800279BB
:106B030008C208C20A8008D2D5790A8004790AC269
:106B1300D5E543047002F543E4FAFDFEFF12697301
:106B2300FC7B08200313126973FD7B1030020A12E9
:106B33006973FE126973FF7B20EC3382D592D550C3
:106B430013C3E43002069FFFE49EFEE42003039D8B
:106B5300FDE49CFCE4CBF8C203EC700CCFCECDCCAF
:106B6300E824F8F870F38017C3EF33FFEE33FEED3C
:106B730033FDEC33FCEB33FB994002FB0FD8E9EB1D
:106B8300300305F8D0E0C448B203C0E00AEC4D4E30
:106B93004F78207B0070C2EAB5430040BCC0E012CE
:106BA3006C08D0F0D0E0200304C4C0E0C4B203C03A
:106BB300F0126997D0F0D5F0EB0269E7126FB26A71
:106BC30084536AFE586A554C6A51426B024F6B0AF2
:0F6BD300446B0A496A6A436B10556AF4466AF4C8
:106BE200456AF4476CB0506A592D6A5D2E6A802B53
:106BF2006A61236A7E206C992A6A194800006A78C1
:106C02003F3F3F00790AA2D5200514300709B91089
:106C1200020404B9080104A2D5200802500104208C
:106C220004689204B542005034C0E07F2030051958
:106C32007F30A20472087207500F126C5FC204C246
:106C420008C207C20A7F30800F300703E9C0E01292
:106C520069AE300703D0E0F9D0E0B542CC30071777
:106C62007F30B9100C1269AE7F583006077F7880EA
:106C720003B908031269AE3004057F2D0269AE7FA5
:106C820020200AF87F2B2008F322920480CF286E5E
:106C9200756C6C2900D2031269733003F8C2037851
:106CA2004230D50108F6026A192D5043495812693B
:106CB200732403B405004001E4906CAB9312699F06
:0D6CC200743A12699FD205754204026AFE01
:10710D008B2E8A2F8930E4F53AF539F538F537F5B8
:10711D0035F536E532453345316012EBC0E0EAC056
:10712D00E0E9C0E0AB31AA32A9331270A3AB2E0552
:10713D0030E530AA2F7002052F14F9126FDEF53BE2
:10714D00C394094007E53BD3940D40E1E53B642032
:10715D0060DBE53BB42D054336038016E53BB42BD0
:10716D0005433601800C74FF2530F53074FF352F43
:10717D00F52FE53460046410703FAB2EAA2FA930B3
:10718D00126FDE64306009E534702E75340A802983
:10719D00900001126FF7FF64786004EFB458134349
:1071AD00360175341074022530F530E4352FF52F86
:1071BD008007E5347003753408AB2E0530E530AA31
:1071CD002F7002052F14F9126FDEF53BC394614049
:1071DD000AE53BD3947A5003533BDF74D0253BF53E
:1071ED003BC3940A400CE53B9411406D74F9253B6B
:1071FD00F53BE53BD395345060433601853A3F85E9
:10720D00393E85383D85373CAF347E00E4FCFDAB1F
:10721D003AAA39A938A837127036C8ECC8C9EDC9D1
:10722D00CAEECACBEFCBE4FCFDFEEB253BF53AEE07
:10723D003AF539ED39F538EC38F537AF3AAE39ADB9
:10724D0038FCAB3FAA3EA93DA83CD3126F4C50036E
:10725D000271C64336040271C6E53620E003E480B0
:10726D002DE53245334531601EAB2EE53024FFF957
:10727D00E52F34FFFAEBC0E0EAC0E0E9C0E0AB3146
:10728D00AA32A9331270A3E53630E20774FFFFFE70
:10729D00FDFC22E536AF3AAE39AD38AC3730E103FF
:0472AD0002708522C4
:106FDE00BB010689828A83E0225002E722BBFE02B1
:096FEE00E32289828A83E49322E4
:106FF700BB010CE58229F582E5833AF583E022504F
:1070070006E92582F8E622BBFE06E92582F8E22298
:0D701700E58229F582E5833AF583E49322B2
:10702400BB010689828A83F0225002F722BBFE014B
:02703400F32245
:10703600E88FF0A4CC8BF0A42CFCE98EF0A42CFCF9
:107046008AF0EDA42CFCEA8EF0A4CDA8F08BF0A477
:107056002DCC3825F0FDE98FF0A42CCD35F0FCEBD6
:107066008EF0A4FEA9F0EB8FF0A4CFC5F02ECD399B
:0F707600FEE43CFCEAA42DCE35F0FDE43CFC2208
:0E708500C3E49FFFE49EFEE49DFDE49CFC221C
:10709300FAE6FB0808E6F925F0F618E6CA3AF622FE
:1070A300BB011A89828A83D0F0D0E0F8D0E0F9D00E
:1070B300E0FAD0E0FBE8C0E0C0F00270FB5016E954
:1070C300F8D083D082D0E0F9D0E0FAD0E0FBC082E0
:1070D300C0830270F2BBFE16E9F8D083D082D0E001
:0F70E300F9D0E0FAD0E0FBC082C0830271042232
:0970F200EBF608EAF608E9F622C3
:0970FB00EBF0A3EAF0A3E9F02296
:09710400EBF208EAF208E9F222BC
:00000001FF
